:2000000021C03AC039C038C037C036C0DDC134C033C032C031C012C52FC02EC02DC02CC032
:200020002BC02AC0C5C693C6B2C626C025C024C023C022C060C524C545C55DC564C5B3C540
:20004000C2C5D6C511241FBECFEFD2E0DEBFCDBF11E0A0E0B1E0E8E6FEE002C005900D922F
:20006000A030B107D9F711E0A0E0B1E001C01D92A030B107E1F701C0C3CFCDEFD2E0DEBFF8
:20008000CDBF14BE88E10FB6F89480936000109260000FBE579A1A82198289819A818F5FCB
:2000A0009F4F31F089819A8101969A838983F5CF4E9901C02AC799D1A7D17894A0E0B0E0F1
:2000C000CBD6802D992780939101809191018F3F19F485E08093910115D25F9A41E18091D2
:2000E000AC018823E1F31092AC011092AD011092DF0190E04093DE019093DD011A9BFECF0E
:20010000409A1A99FECF83E184B980E48CBD1DBC0DB40EB440988091E501882309F445C05F
:200120001092E5018091E701882349F11092E7018091020180FF0CC08091020182FF2BC0F0
:200140008091020181FF23C08091DF0182600BC08091020181FF17C08091020182FF1FC0AB
:200160008091DF0181608093DF018091DF0184608093DF0192E882E28093DE0118C0809139
:20018000020180FF08C08091020182FF0EC08091DF01826007C08091020181FF06C08091AD
:2001A000DF0181608093DF0192E04093DE018091E601882341F01092E60198608091DF0121
:2001C00088608093DF018091E801882331F098608091DF0180618093DF019EBD429A0DB4C9
:2001E00007FEFDCF1A99A3C042988091AD01873198F48091DC01882339F08091AD01E82FA3
:20020000FF27E255FE4F06C08091AD01E82FFF27EB53FE4F8EB580838091AD018F5F8093E1
:20022000AD019091DD01992309F043C08091DF0182FF1CC08091DF0180FF0CC08091AD0110
:20024000823120F18091AD01E82FFF27E850FF4F808123C08091AD01823160F08091AD01F3
:20026000E82FFF27E050FF4F878517C08091DF0180FF08C08091AD01E82FFF27E050FF4F2E
:2002800081850BC08091DF0181FF09C08091AD01E82FFF27E050FF4F80A18EBD01C09EBD51
:2002A0009091AD018091DE01981709F03FC081E03BC08091DD01813031F58091DF0183FF43
:2002C00014C08091DF0182FF07C08091AD01E82FFF27ED51FF4F06C08091AD01E82FFF27C7
:2002E000EC50FF4F80818EBD01C01EBC8091AD01282F33278091DE01992704962817390754
:20030000A9F482E011C08091DD01823081F48091E8019091E401892B8EBD8091E80181304D
:2003200011F01092E80183E08093DD01429A0DB407FEFDCF8091DD01833009F053CF4298D8
:200340008091AD018731A0F58091DC018823B9F08091AD01E82FFF27E255FE4F8EB5808389
:200360008091AE0183FF24C0A0EEB1E0E0ECF1E094E081918D93915097FFFBCF16C08091CD
:20038000AD01E82FFF27EB53FE4F8EB580838091C50183FF0DC0A0EEB1E0E7EDF1E094E043
:2003A00081918D93915097FFFBCF80E88093E40190E08091DC01882309F491E09093DC01F3
:2003C0001CBC83E084B98BCE1F920F920FB60F9211248F93809160008F7B809360008F912F
:2003E0000F900FBE0F901F90189590E395B983E084B998B98FE087B980E48BB986EA8AB9DA
:2004000085E08093C40008958DB78095E0E0F1E02FEF32E0281B3109E217F30710F41192D2
:20042000FBCF109290011092A60181E08093A7011092AC011092DC011092E5011092E6017B
:200440001092E7011092E8011092E9011092EA011092850196E3909381019093820190935F
:20046000830125E52093420180914201809341018091410180934001209345018091450158
:200480008093440180914401809343018FEF8093470180914701809346018091870180931F
:2004A00048019093490190934A0190934B0187E080934C0182E080934D0110924E0120937B
:2004C0004F0120935001209351010FD0089520E0281750F49FE00000000000000000915064
:2004E00097FFF9CF2F5FF4CF0895ECE4F1E020E090914C01923020F0819128279150FACFC4
:20050000208308950F931F93CF9300E0009387014AD284E0DCDF80918701815E809387019C
:2005200080918701853610F010928701809187018093800160E0809187013ED2549885E2D4
:20054000C6DF5D9A85E0C3DF10928D011092C00080E98093C10086E48093C200E8D380911E
:200560008C018F3F89F5C0918D01CC2369F510910101113049F55AD2C0938C0180918601B0
:20058000806880938601209184003091850080918E0190918F01281B390B83E0220F331FA0
:2005A0008A95E1F78AE094E0821B930B9093890080938800AFD380910301809382018093A4
:2005C0004A0134D2012F07C08091840090918500815C984A20F21092C200002309F498CFDC
:2005E000809190018823E1F3109290018091010180FFF6CF8091010182FFF2CF80914D019C
:20060000846080934D0171DF809190018823E1F3109290018091010180FFF6CF8091010187
:2006200082FFF2CF84E380934C019FEFE2E5F1E083E09193815087FFFCCF95E5E6E5F1E0CC
:2006400088E29193815087FFFCCF4FDF80918601806180938601CF911F910F91089580914B
:20066000860185FF54C180919001882339F18091010183FF23C01092900180910301809310
:20068000AA01809104018093AB018091AA018431A8F48091AB018F3588F48091AA019091F3
:2006A000AB01890F90910501891741F480914D01806180934D0180E28093A70180914E01DC
:2006C00080FF31C080914E0182FF04C084E080934E0102C010924E018091DC01882381F47E
:2006E0008091AE0181FF50C0AFEAB1E0E1E4F1E090E18D91858B9150319697FFFACF0FC075
:200700008091C50181FF40C0A6ECB1E0E1E4F1E090E18D91858B9150319697FFFACF809112
:200720004E0182602FC080914E0181FF02C083E001C081E080934E018091DC01882381F402
:200740008091AE0181FF20C0AFEAB1E0E1E4F1E090E18D9184A79150319697FFFACF0FC029
:200760008091C50181FF10C0A6ECB1E0E1E4F1E090E18D9184A79150319697FFFACF8091C7
:200780004E01846080934E018091850187FF81C080918501803841F52091E801222321F5EC
:2007A0008091F00E809352019091F10E892F807E809353019F7180915301892B80935301F7
:2007C0008091F20E809354018091F30E8093550180914E01886080934E012093E90181E07D
:2007E0008093E80181E827C080918501813831F52091E801222311F58091F40E80935201D9
:200800008091F50E9091F60E892F9927809353018091F50E809354018091F70E80935501C5
:2008200080914E01886080934E012093E90181E08093E80182E88093850149C08091850171
:20084000823809F044C02091E801222309F03FC08091F80E809352018091F90E9091FA0E4C
:20086000892F9927809353018091F90E809354018091FB0E8093550180914E01886080933B
:200880004E012093E90181E08093E801209385011EC08091E4018823D1F08091E8018823F1
:2008A000B1F48093E401A0EEB1E0E2E5F1E093E08D918193915097FFFBCF80914E018860B6
:2008C00080934E011092E90181E08093E8018091E801813091F48091E901893121F483E070
:2008E0008093E8010AC080914E01886080934E018091E9018F5F8093E9018091EA018823FB
:2009000089F180914E01806880934E012BC08091A70181FF10C080919001882309F442C073
:2009200010929001809105018F5F8093A80184E08093A70108958091A70182FF15C08091E7
:20094000A8018F5F8093A8018091A80184FF2AC08091860180628093860180914D018F7E9D
:2009600080934D01C2DD08958091A70180FF1AC08091010183FF16C0E0E0F1E0A2E9B1E0B0
:2009800093E186818D939150319697FFFACF80914D01806180934D01A8DD1092900182E0FA
:2009A0008093A7010895299A5A9A419A5D9828985C985998549A0895982F299A59985C98B9
:2009C000419834E360FF0BC080919101880F80939101309191013167892F855E0FC0892F11
:2009E000845E20EA98E05C9827FF02C0599A01C05998220F5C9A915097FFF5CF8068232F76
:200A00003327322F2227280F311D9FE05C9837FF02C0599A01C05998220F331F5C9A9150E3
:200A200097FFF4CF5C985998419A08955D98289829985A9841985C98599808951F920F92EB
:200A40000FB60F9211242F933F934F935F936F937F938F939F93AF93BF93CF93EF93FF9321
:200A6000C0918801CF5F8C2F9927AA27BB27FC013197E830F10508F039C1E65EFF4F09944C
:200A800061E08091870198DF80E48093C00088E08093C100809188009091890085599E4F84
:200AA000909389008093880080918701809348018091860184FDD3DD80914C01845F8093DD
:200AC000890114C18091880090918900805F9A4F909389008093880010928A0186E48093BB
:200AE000C200289A88E28093C10085E58093C6008093C600FBC057DF8091880090918900E4
:200B00008B5B9F4F70C08091860185FF29C08091A601E82FFF27EE56FE4F808180938701AA
:200B20008091A6018F5F8093A6018091A601843111F51092A6018091A70185FF1CC01092DE
:200B4000A7018091AA01E82FFF27EE56FE4F8091AB01808380914D018F7E80934D010BC00B
:200B600080918701815E8093870180918701853610F01092870110928B0110928C011092E5
:200B8000900110928D0160E08091870115DF80918800909189008C5E9E4F909389008093EE
:200BA00088005498A3C08091880090918900895A9F4F90938900809388005D9A8091870173
:200BC0008093800193C010928D011092C00080E98093C10086E48093C20080918800909166
:200BE00089008C599B4F90938900809388007EC01092C0001092C1001092C20017DFC0E059
:200C000080918C018F3F09F04EC080918D01882309F049C080918E0190918F01815F9B4FFA
:200C2000909389008093880021E02093900188B198E0892788B9C093EB018091020180FFB4
:200C400005C08091020182FD09C004C08091020181FD04C08091E701882311F02093E5011B
:200C60008091020183FF11C08091EA01882399F480910601843019F480E88093850181E09E
:200C80008093E6018093EA0106C08091EA01882311F01092EA018091020187FF20C082E085
:200CA0008093E8011CC0809188009091890084559F4F909389008093880081E08093E701AF
:200CC0008091860184FF0BC08091EB018F5F8093EB018091EB018F3F11F45F98B0D08091EC
:200CE000860185FF03C081E08093AC01C0938801FF91EF91CF91BF91AF919F918F917F91C9
:200D00006F915F914F913F912F910F900FBE0F901F9018951092850010928400109280009D
:200D200082E08093810080936F0086BB08951092850010928400109280001092820082E068
:200D400086BB10926F0083E0809381000895DEBBDFB7DABDCBBDD1E0C0918A01C05CD8815D
:200D6000D093C600CF53C0938A01C83009F42998D0918901DC1731F4D0E4D093C000D8E4FE
:200D8000D093C100CBB5DAB5DFBFDEB31895DEBBDFB7DABDD0E0D093C000D093C100D09324
:200DA000C2005A9828984198DAB5DFBFDEB318959EBBEABDFBBDFFB7F8BD90918C019430E6
:200DC000B1F0E0E8F1E0E90FF081E091C600FE1771F5939590938C01943059F5E0918400DF
:200DE000E0938E01E0918500E0938F0122C09091C600F1E0E0918B019083E395EF73E09301
:200E00008B01F0918D01F927F0938D01909100019E1779F49FEF90938C0190E09093C10030
:200E20009093C2005A985D984198299802C010928C01F8B5FFBFFBB5EAB59EB31895A89566
:200E400088E190E028E00FB6F894A895809360000FBE20936000FFCFF999FECFB2BDA1BDD6
:200E6000F89A119600B40895FFFFFFFFFFFFFFFFFFFFFFFFFFFFFFFFFFFFFFFFFFFFFFFF00
:200E80000FEFFFFFFFFFFFFFFFFFFFFFFFFFFFFFFFFFFFFFFFFFFFFFFFFFFFFFFFFFFFFF72
:200EA0000FEFFFFFFFFFFFFFFFFFFFFFFFFFFFFFFFFFFFFFFFFFFFFFFFFFFFFFFFFFFFFF52
:200EC0000FEFFFFFFFFFFFFFFFFFFFFFFFFFFFFFFFFFFFFFFFFFFFFFFFFFFFFFFFFFFFFF32
:200EE0000FEFFFFFFFFFFFFFFFFFFFFFFFFFFFFFC8020300C9EEFF00CA000000FFFFFFFFB9
:200F00008091BC008823E4F7089500E010E068018DE38093B80084E68093BA0084EC8093B3
:200F2000BC00EEDF8091B900887F803609F0FFCF84EC8093BC00E4DF8091B900887F80384F
:200F400009F0FFCF8091BB00182F84EC8093BC00D7DF8091B900887F803809F0FFCF809161
:200F6000BB00082FC8018F739070892B09F0FFCF8FE00030180708F0FFCFE80184EC809349
:200F8000BC00EE24FF248FE3B82EBADF8091B900887F803891F4E0FC04C08091BB00C82EFF
:200FA0000DC08091BB00D82E81E00601FE0180935700E8951124229601C0FFCF84EC809345
:200FC000BC00BA940894E11CF11CB7FEDECF98DF8091B900887F803A09F0FFCF84EC8093B3
:180FE000BC0083E0F80180935700E89585E0F80180935700E89595CF51
:00000001FF
